 ForceEarlyReturnTest

 Timestamp is 2d246ee3 (reproducible build file hash)

 Preferred load address is 0000000180000000

 Start         Length     Name                   Class
 0001:00000000 00001a80H .text$mn                CODE
 0001:00001a80 00000036H .text$mn$00             CODE
 0001:00001ab6 00000092H .text$x                 CODE
 0002:00000000 00000158H .idata$5                DATA
 0002:00000158 00000038H .00cfg                  DATA
 0002:00000190 00000008H .CRT$XCA                DATA
 0002:00000198 00000008H .CRT$XCZ                DATA
 0002:000001a0 00000008H .CRT$XIA                DATA
 0002:000001a8 00000008H .CRT$XIC                DATA
 0002:000001b0 00000008H .CRT$XIZ                DATA
 0002:000001b8 00000008H .CRT$XLA                DATA
 0002:000001c0 00000008H .CRT$XLZ                DATA
 0002:000001c8 00000008H .CRT$XPA                DATA
 0002:000001d0 00000008H .CRT$XPZ                DATA
 0002:000001d8 00000008H .CRT$XTA                DATA
 0002:000001e0 00000010H .CRT$XTZ                DATA
 0002:000001e8 00000000H .gehcont$y              DATA
 0002:000001e8 00000000H .gfids$y                DATA
 0002:000001f0 00001090H .rdata                  DATA
 0002:00001280 00000000H .rdata$CastGuardVftablesA DATA
 0002:00001280 00000000H .rdata$CastGuardVftablesC DATA
 0002:00001280 00000028H .rdata$T                DATA
 0002:000012a8 00000070H .rdata$voltmd           DATA
 0002:00001318 00000328H .rdata$zzzdbg           DATA
 0002:00001640 00000008H .rtc$IAA                DATA
 0002:00001648 00000008H .rtc$IZZ                DATA
 0002:00001650 00000008H .rtc$TAA                DATA
 0002:00001658 00000008H .rtc$TZZ                DATA
 0002:00001660 00000004H .tls                    DATA
 0002:00001664 00000004H .tls$                   DATA
 0002:00001668 00000008H .tls$ZZZ                DATA
 0002:00001670 000001c0H .xdata                  DATA
 0002:00001830 000001fcH .edata                  DATA
 0002:00001a2c 00000050H .idata$2                DATA
 0002:00001a7c 00000014H .idata$3                DATA
 0002:00001a90 00000158H .idata$4                DATA
 0002:00001be8 000003a6H .idata$6                DATA
 0003:00000000 00000050H .data                   DATA
 0003:00000050 000007b8H .bss                    DATA
 0004:00000000 0000027cH .pdata                  DATA

  Address         Publics by Value              Rva+Base               Lib:Object

 0000:00000000       __AbsoluteZero             0000000000000000     <absolute>
 0000:00000000       ___safe_se_handler_count   0000000000000000     <absolute>
 0000:00000000       ___safe_se_handler_table   0000000000000000     <absolute>
 0000:00000000       __arm64x_extra_rfe_table   0000000000000000     <absolute>
 0000:00000000       __arm64x_extra_rfe_table_size 0000000000000000     <absolute>
 0000:00000000       __arm64x_native_entrypoint 0000000000000000     <absolute>
 0000:00000000       __arm64x_redirection_metadata 0000000000000000     <absolute>
 0000:00000000       __arm64x_redirection_metadata_count 0000000000000000     <absolute>
 0000:00000000       __dynamic_value_reloc_table 0000000000000000     <absolute>
 0000:00000000       __enclave_config           0000000000000000     <absolute>
 0000:00000000       __guard_check_icall_a64n_fptr 0000000000000000     <absolute>
 0000:00000000       __guard_eh_cont_count      0000000000000000     <absolute>
 0000:00000000       __guard_eh_cont_table      0000000000000000     <absolute>
 0000:00000000       __guard_fids_count         0000000000000000     <absolute>
 0000:00000000       __guard_fids_table         0000000000000000     <absolute>
 0000:00000000       __guard_iat_count          0000000000000000     <absolute>
 0000:00000000       __guard_iat_table          0000000000000000     <absolute>
 0000:00000000       __guard_longjmp_count      0000000000000000     <absolute>
 0000:00000000       __guard_longjmp_table      0000000000000000     <absolute>
 0000:00000000       __hybrid_auxiliary_iat     0000000000000000     <absolute>
 0000:00000000       __hybrid_auxiliary_iat_copy 0000000000000000     <absolute>
 0000:00000000       __hybrid_code_map          0000000000000000     <absolute>
 0000:00000000       __hybrid_code_map_count    0000000000000000     <absolute>
 0000:00000000       __x64_code_ranges_to_entry_points 0000000000000000     <absolute>
 0000:00000000       __x64_code_ranges_to_entry_points_count 0000000000000000     <absolute>
 0000:00000100       __guard_flags              0000000000000100     <absolute>
 0000:00000000       __ImageBase                0000000180000000     <linker-defined>
 0001:00000000       ?SetEventNotificationMode@_jvmtiEnv@@QEAA?AW4jvmtiError@@W4jvmtiEventMode@@W4jvmtiEvent@@PEAV_jobject@@ZZ 0000000180001000 f i libForceEarlyReturnTest.obj
 0001:0000000c       ?TranslateError@@YAPEBDW4jvmtiError@@@Z 000000018000100c f   libForceEarlyReturnTest.obj
 0001:0000032c       ?create_raw_monitor@@YAPEAU_jrawMonitorID@@PEAU_jvmtiEnv@@PEBD@Z 000000018000132c f   libForceEarlyReturnTest.obj
 0001:00000358       Agent_Initialize           0000000180001358 f   libForceEarlyReturnTest.obj
 0001:000004fc       Agent_OnLoad               00000001800014fc f   libForceEarlyReturnTest.obj
 0001:00000748       Java_ForceEarlyReturnTest_ensureAtBreakpoint 0000000180001748 f   libForceEarlyReturnTest.obj
 0001:00000800       Java_ForceEarlyReturnTest_forceEarlyReturnI 0000000180001800 f   libForceEarlyReturnTest.obj
 0001:00000858       Java_ForceEarlyReturnTest_forceEarlyReturnO 0000000180001858 f   libForceEarlyReturnTest.obj
 0001:000008b0       Java_ForceEarlyReturnTest_forceEarlyReturnV 00000001800018b0 f   libForceEarlyReturnTest.obj
 0001:00000904       Java_ForceEarlyReturnTest_notifyAtBreakpoint 0000000180001904 f   libForceEarlyReturnTest.obj
 0001:000009c8       Java_ForceEarlyReturnTest_prepareAgent 00000001800019c8 f   libForceEarlyReturnTest.obj
 0001:00000acc       Java_ForceEarlyReturnTest_resumeThread 0000000180001acc f   libForceEarlyReturnTest.obj
 0001:00000b2c       Java_ForceEarlyReturnTest_suspendThread 0000000180001b2c f   libForceEarlyReturnTest.obj
 0001:00000b8c       __local_stdio_printf_options 0000000180001b8c f i libForceEarlyReturnTest.obj
 0001:00000b94       printf                     0000000180001b94 f i libForceEarlyReturnTest.obj
 0001:00000cf0       __security_check_cookie    0000000180001cf0 f   MSVCRT:amdsecgs.obj
 0001:00001030       _DllMainCRTStartup         0000000180002030 f   MSVCRT:dll_dllmain.obj
 0001:00001070       __scrt_acquire_startup_lock 0000000180002070 f   MSVCRT:utility.obj
 0001:000010ac       __scrt_dllmain_after_initialize_c 00000001800020ac f   MSVCRT:utility.obj
 0001:000010e0       __scrt_dllmain_before_initialize_c 00000001800020e0 f   MSVCRT:utility.obj
 0001:000010f8       __scrt_dllmain_crt_thread_attach 00000001800020f8 f   MSVCRT:utility.obj
 0001:00001120       __scrt_dllmain_crt_thread_detach 0000000180002120 f   MSVCRT:utility.obj
 0001:00001138       __scrt_dllmain_exception_filter 0000000180002138 f   MSVCRT:utility.obj
 0001:00001198       __scrt_dllmain_uninitialize_c 0000000180002198 f   MSVCRT:utility.obj
 0001:000011c8       __scrt_dllmain_uninitialize_critical 00000001800021c8 f   MSVCRT:utility.obj
 0001:000011dc       __scrt_initialize_crt      00000001800021dc f   MSVCRT:utility.obj
 0001:00001228       __scrt_initialize_onexit_tables 0000000180002228 f   MSVCRT:utility.obj
 0001:000012b4       __scrt_is_nonwritable_in_current_image 00000001800022b4 f   MSVCRT:utility.obj
 0001:0000134c       __scrt_release_startup_lock 000000018000234c f   MSVCRT:utility.obj
 0001:00001370       __scrt_uninitialize_crt    0000000180002370 f   MSVCRT:utility.obj
 0001:0000139c       _onexit                    000000018000239c f   MSVCRT:utility.obj
 0001:000013d8       atexit                     00000001800023d8 f   MSVCRT:utility.obj
 0001:000013f0       __crt_debugger_hook        00000001800023f0 f   MSVCRT:utility_desktop.obj
 0001:000013f8       __scrt_fastfail            00000001800023f8 f   MSVCRT:utility_desktop.obj
 0001:00001544       _guard_check_icall_nop     0000000180002544 f i MSVCRT:guard_support.obj
 0001:00001548       __raise_securityfailure    0000000180002548 f   MSVCRT:gs_report.obj
 0001:0000157c       __report_gsfailure         000000018000257c f   MSVCRT:gs_report.obj
 0001:000016c4       __security_init_cookie     00000001800026c4 f   MSVCRT:gs_support.obj
 0001:00001770       DllMain                    0000000180002770 f   MSVCRT:dll_dllmain_stub.obj
 0001:00001794       ?__scrt_initialize_type_info@@YAXXZ 0000000180002794 f   MSVCRT:tncleanup.obj
 0001:000017a4       ?__scrt_uninitialize_type_info@@YAXXZ 00000001800027a4 f   MSVCRT:tncleanup.obj
 0001:000017b0       __local_stdio_scanf_options 00000001800027b0 f i MSVCRT:default_local_stdio_options.obj
 0001:000017b8       __scrt_initialize_default_local_stdio_options 00000001800027b8 f   MSVCRT:default_local_stdio_options.obj
 0001:000017d4       __scrt_get_dyn_tls_init_callback 00000001800027d4 f   MSVCRT:dyn_tls_init.obj
 0001:000017dc       _RTC_Initialize            00000001800027dc f   MSVCRT:initsect.obj
 0001:00001818       _RTC_Terminate             0000000180002818 f   MSVCRT:initsect.obj
 0001:00001854       __isa_available_init       0000000180002854 f   MSVCRT:cpu_disp.obj
 0001:00001a00       _get_startup_argv_mode     0000000180002a00 f   MSVCRT:argv_mode.obj
 0001:00001a08       __scrt_is_ucrt_dll_in_use  0000000180002a08 f   MSVCRT:ucrt_detection.obj
 0001:00001a20       __C_specific_handler       0000000180002a20 f   vcruntime:VCRUNTIME140.dll
 0001:00001a26       memset                     0000000180002a26 f   vcruntime:VCRUNTIME140.dll
 0001:00001a2c       __std_type_info_destroy_list 0000000180002a2c f   vcruntime:VCRUNTIME140.dll
 0001:00001a32       _initterm                  0000000180002a32 f   ucrt:api-ms-win-crt-runtime-l1-1-0.dll
 0001:00001a38       _initterm_e                0000000180002a38 f   ucrt:api-ms-win-crt-runtime-l1-1-0.dll
 0001:00001a3e       _seh_filter_dll            0000000180002a3e f   ucrt:api-ms-win-crt-runtime-l1-1-0.dll
 0001:00001a44       _configure_narrow_argv     0000000180002a44 f   ucrt:api-ms-win-crt-runtime-l1-1-0.dll
 0001:00001a4a       _initialize_narrow_environment 0000000180002a4a f   ucrt:api-ms-win-crt-runtime-l1-1-0.dll
 0001:00001a50       _initialize_onexit_table   0000000180002a50 f   ucrt:api-ms-win-crt-runtime-l1-1-0.dll
 0001:00001a56       _register_onexit_function  0000000180002a56 f   ucrt:api-ms-win-crt-runtime-l1-1-0.dll
 0001:00001a5c       _execute_onexit_table      0000000180002a5c f   ucrt:api-ms-win-crt-runtime-l1-1-0.dll
 0001:00001a62       _crt_atexit                0000000180002a62 f   ucrt:api-ms-win-crt-runtime-l1-1-0.dll
 0001:00001a68       _cexit                     0000000180002a68 f   ucrt:api-ms-win-crt-runtime-l1-1-0.dll
 0001:00001a70       __acrt_initialize          0000000180002a70 f   MSVCRT:ucrt_stubs.obj
 0001:00001a70       __acrt_thread_attach       0000000180002a70 f   MSVCRT:ucrt_stubs.obj
 0001:00001a70       __acrt_thread_detach       0000000180002a70 f   MSVCRT:ucrt_stubs.obj
 0001:00001a70       __acrt_uninitialize        0000000180002a70 f   MSVCRT:ucrt_stubs.obj
 0001:00001a70       __acrt_uninitialize_critical 0000000180002a70 f   MSVCRT:ucrt_stubs.obj
 0001:00001a70       __scrt_stub_for_acrt_initialize 0000000180002a70 f   MSVCRT:ucrt_stubs.obj
 0001:00001a70       __scrt_stub_for_acrt_thread_attach 0000000180002a70 f   MSVCRT:ucrt_stubs.obj
 0001:00001a70       __scrt_stub_for_acrt_thread_detach 0000000180002a70 f   MSVCRT:ucrt_stubs.obj
 0001:00001a70       __scrt_stub_for_acrt_uninitialize 0000000180002a70 f   MSVCRT:ucrt_stubs.obj
 0001:00001a70       __scrt_stub_for_acrt_uninitialize_critical 0000000180002a70 f   MSVCRT:ucrt_stubs.obj
 0001:00001a70       __vcrt_initialize          0000000180002a70 f   MSVCRT:ucrt_stubs.obj
 0001:00001a70       __vcrt_thread_attach       0000000180002a70 f   MSVCRT:ucrt_stubs.obj
 0001:00001a70       __vcrt_thread_detach       0000000180002a70 f   MSVCRT:ucrt_stubs.obj
 0001:00001a70       __vcrt_uninitialize        0000000180002a70 f   MSVCRT:ucrt_stubs.obj
 0001:00001a70       __vcrt_uninitialize_critical 0000000180002a70 f   MSVCRT:ucrt_stubs.obj
 0001:00001a74       __scrt_stub_for_is_c_termination_complete 0000000180002a74 f   MSVCRT:ucrt_stubs.obj
 0001:00001a74       _is_c_termination_complete 0000000180002a74 f   MSVCRT:ucrt_stubs.obj
 0001:00001a77       memcpy                     0000000180002a77 f   vcruntime:VCRUNTIME140.dll
 0001:00001a90       _guard_dispatch_icall_nop  0000000180002a90 f   MSVCRT:guard_dispatch.obj
 0001:00001ab0       _guard_xfg_dispatch_icall_nop 0000000180002ab0 f   MSVCRT:guard_xfg_dispatch.obj
 0002:00000000       __imp_Sleep                0000000180003000     kernel32:KERNEL32.dll
 0002:00000008       __imp_CloseHandle          0000000180003008     kernel32:KERNEL32.dll
 0002:00000010       __imp_InitializeCriticalSectionAndSpinCount 0000000180003010     kernel32:KERNEL32.dll
 0002:00000018       __imp_DeleteCriticalSection 0000000180003018     kernel32:KERNEL32.dll
 0002:00000020       __imp_CreateEventW         0000000180003020     kernel32:KERNEL32.dll
 0002:00000028       __imp_GetModuleHandleW     0000000180003028     kernel32:KERNEL32.dll
 0002:00000030       __imp_GetProcAddress       0000000180003030     kernel32:KERNEL32.dll
 0002:00000038       __imp_RtlCaptureContext    0000000180003038     kernel32:KERNEL32.dll
 0002:00000040       __imp_RtlLookupFunctionEntry 0000000180003040     kernel32:KERNEL32.dll
 0002:00000048       __imp_RtlVirtualUnwind     0000000180003048     kernel32:KERNEL32.dll
 0002:00000050       __imp_IsDebuggerPresent    0000000180003050     kernel32:KERNEL32.dll
 0002:00000058       __imp_UnhandledExceptionFilter 0000000180003058     kernel32:KERNEL32.dll
 0002:00000060       __imp_SetUnhandledExceptionFilter 0000000180003060     kernel32:KERNEL32.dll
 0002:00000068       __imp_IsProcessorFeaturePresent 0000000180003068     kernel32:KERNEL32.dll
 0002:00000070       __imp_GetCurrentProcess    0000000180003070     kernel32:KERNEL32.dll
 0002:00000078       __imp_TerminateProcess     0000000180003078     kernel32:KERNEL32.dll
 0002:00000080       __imp_QueryPerformanceCounter 0000000180003080     kernel32:KERNEL32.dll
 0002:00000088       __imp_GetCurrentProcessId  0000000180003088     kernel32:KERNEL32.dll
 0002:00000090       __imp_GetCurrentThreadId   0000000180003090     kernel32:KERNEL32.dll
 0002:00000098       __imp_GetSystemTimeAsFileTime 0000000180003098     kernel32:KERNEL32.dll
 0002:000000a0       __imp_DisableThreadLibraryCalls 00000001800030a0     kernel32:KERNEL32.dll
 0002:000000a8       __imp_InitializeSListHead  00000001800030a8     kernel32:KERNEL32.dll
 0002:000000b0       \177KERNEL32_NULL_THUNK_DATA 00000001800030b0     kernel32:KERNEL32.dll
 0002:000000b8       __imp___C_specific_handler 00000001800030b8     vcruntime:VCRUNTIME140.dll
 0002:000000c0       __imp_memset               00000001800030c0     vcruntime:VCRUNTIME140.dll
 0002:000000c8       __imp___std_type_info_destroy_list 00000001800030c8     vcruntime:VCRUNTIME140.dll
 0002:000000d0       __imp_memcpy               00000001800030d0     vcruntime:VCRUNTIME140.dll
 0002:000000d8       \177VCRUNTIME140_NULL_THUNK_DATA 00000001800030d8     vcruntime:VCRUNTIME140.dll
 0002:000000e0       __imp__initialize_onexit_table 00000001800030e0     ucrt:api-ms-win-crt-runtime-l1-1-0.dll
 0002:000000e8       __imp__cexit               00000001800030e8     ucrt:api-ms-win-crt-runtime-l1-1-0.dll
 0002:000000f0       __imp__crt_atexit          00000001800030f0     ucrt:api-ms-win-crt-runtime-l1-1-0.dll
 0002:000000f8       __imp__execute_onexit_table 00000001800030f8     ucrt:api-ms-win-crt-runtime-l1-1-0.dll
 0002:00000100       __imp__initterm            0000000180003100     ucrt:api-ms-win-crt-runtime-l1-1-0.dll
 0002:00000108       __imp__initterm_e          0000000180003108     ucrt:api-ms-win-crt-runtime-l1-1-0.dll
 0002:00000110       __imp__seh_filter_dll      0000000180003110     ucrt:api-ms-win-crt-runtime-l1-1-0.dll
 0002:00000118       __imp__configure_narrow_argv 0000000180003118     ucrt:api-ms-win-crt-runtime-l1-1-0.dll
 0002:00000120       __imp__register_onexit_function 0000000180003120     ucrt:api-ms-win-crt-runtime-l1-1-0.dll
 0002:00000128       __imp__initialize_narrow_environment 0000000180003128     ucrt:api-ms-win-crt-runtime-l1-1-0.dll
 0002:00000130       \177api-ms-win-crt-runtime-l1-1-0_NULL_THUNK_DATA 0000000180003130     ucrt:api-ms-win-crt-runtime-l1-1-0.dll
 0002:00000138       __imp___acrt_iob_func      0000000180003138     ucrt:api-ms-win-crt-stdio-l1-1-0.dll
 0002:00000140       __imp___stdio_common_vfprintf 0000000180003140     ucrt:api-ms-win-crt-stdio-l1-1-0.dll
 0002:00000148       __imp_fflush               0000000180003148     ucrt:api-ms-win-crt-stdio-l1-1-0.dll
 0002:00000150       \177api-ms-win-crt-stdio-l1-1-0_NULL_THUNK_DATA 0000000180003150     ucrt:api-ms-win-crt-stdio-l1-1-0.dll
 0002:00000158       __guard_check_icall_fptr   0000000180003158     MSVCRT:guard_support.obj
 0002:00000160       __guard_xfg_check_icall_fptr 0000000180003160     MSVCRT:guard_support.obj
 0002:00000168       __guard_dispatch_icall_fptr 0000000180003168     MSVCRT:guard_support.obj
 0002:00000170       __guard_xfg_dispatch_icall_fptr 0000000180003170     MSVCRT:guard_support.obj
 0002:00000178       __guard_xfg_table_dispatch_icall_fptr 0000000180003178     MSVCRT:guard_support.obj
 0002:00000180       __castguard_check_failure_os_handled_fptr 0000000180003180     MSVCRT:guard_support.obj
 0002:00000188       __guard_memcpy_fptr        0000000180003188     vcruntime:softmemtag.obj
 0002:00000190       __xc_a                     0000000180003190     MSVCRT:initializers.obj
 0002:00000198       __xc_z                     0000000180003198     MSVCRT:initializers.obj
 0002:000001a0       __xi_a                     00000001800031a0     MSVCRT:initializers.obj
 0002:000001b0       __xi_z                     00000001800031b0     MSVCRT:initializers.obj
 0002:000001b8       __xl_a                     00000001800031b8     MSVCRT:tlssup.obj
 0002:000001c0       __xl_z                     00000001800031c0     MSVCRT:tlssup.obj
 0002:000001c8       __xp_a                     00000001800031c8     MSVCRT:initializers.obj
 0002:000001d0       __xp_z                     00000001800031d0     MSVCRT:initializers.obj
 0002:000001d8       __xt_a                     00000001800031d8     MSVCRT:initializers.obj
 0002:000001e0       __xt_z                     00000001800031e0     MSVCRT:initializers.obj
 0002:000001f0       ??_C@_0DM@KLJPMIDM@check_jvmti_status?3?5JVMTI?5funct@ 00000001800031f0     libForceEarlyReturnTest.obj
 0002:00000230       ??_C@_0CA@CCEFGCFD@Fatal?5Error?5in?5RawMonitorEnter?4@ 0000000180003230     libForceEarlyReturnTest.obj
 0002:00000250       ??_C@_0BP@POHFIHGF@Fatal?5Error?5in?5RawMonitorWait?4@ 0000000180003250     libForceEarlyReturnTest.obj
 0002:00000270       ??_C@_0CE@INHKDOCL@Fatal?5Error?5in?5RawMonitorNotify@ 0000000180003270     libForceEarlyReturnTest.obj
 0002:00000298       ??_C@_0BN@DPBGGNAC@error?5in?5JVMTI?5SuspendThread@ 0000000180003298     libForceEarlyReturnTest.obj
 0002:000002b8       ??_C@_0BM@HOJKOFIM@error?5in?5JVMTI?5ResumeThread@ 00000001800032b8     libForceEarlyReturnTest.obj
 0002:000002d8       ??_C@_0BB@JCNMKLLK@JVMTI_ERROR_NONE@ 00000001800032d8     libForceEarlyReturnTest.obj
 0002:000002f0       ??_C@_0BL@LDIMKLPH@JVMTI_ERROR_INVALID_THREAD@ 00000001800032f0     libForceEarlyReturnTest.obj
 0002:00000310       ??_C@_0CB@PJFPAIKJ@JVMTI_ERROR_INVALID_THREAD_GROU@ 0000000180003310     libForceEarlyReturnTest.obj
 0002:00000338       ??_C@_0BN@LLMKHMNF@JVMTI_ERROR_INVALID_PRIORITY@ 0000000180003338     libForceEarlyReturnTest.obj
 0002:00000358       ??_C@_0CB@MBOFKAGB@JVMTI_ERROR_THREAD_NOT_SUSPENDE@ 0000000180003358     libForceEarlyReturnTest.obj
 0002:00000380       ??_C@_0BN@FABOLPBI@JVMTI_ERROR_THREAD_SUSPENDED@ 0000000180003380     libForceEarlyReturnTest.obj
 0002:000003a0       ??_C@_0BN@FDGNOBJM@JVMTI_ERROR_THREAD_NOT_ALIVE@ 00000001800033a0     libForceEarlyReturnTest.obj
 0002:000003c0       ??_C@_0BL@GOBIFKNJ@JVMTI_ERROR_INVALID_OBJECT@ 00000001800033c0     libForceEarlyReturnTest.obj
 0002:000003e0       ??_C@_0BK@FCMAJPPC@JVMTI_ERROR_INVALID_CLASS@ 00000001800033e0     libForceEarlyReturnTest.obj
 0002:00000400       ??_C@_0BP@IKLLBKEB@JVMTI_ERROR_CLASS_NOT_PREPARED@ 0000000180003400     libForceEarlyReturnTest.obj
 0002:00000420       ??_C@_0BN@KLPPLKG@JVMTI_ERROR_INVALID_METHODID@ 0000000180003420     libForceEarlyReturnTest.obj
 0002:00000440       ??_C@_0BN@BCEKOKND@JVMTI_ERROR_INVALID_LOCATION@ 0000000180003440     libForceEarlyReturnTest.obj
 0002:00000460       ??_C@_0BM@DFDGPME@JVMTI_ERROR_INVALID_FIELDID@ 0000000180003460     libForceEarlyReturnTest.obj
 0002:00000480       ??_C@_0BL@NELIEPEC@JVMTI_ERROR_NO_MORE_FRAMES@ 0000000180003480     libForceEarlyReturnTest.obj
 0002:000004a0       ??_C@_0BJ@BDBECFDM@JVMTI_ERROR_OPAQUE_FRAME@ 00000001800034a0     libForceEarlyReturnTest.obj
 0002:000004c0       ??_C@_0BK@MIIFNLOB@JVMTI_ERROR_TYPE_MISMATCH@ 00000001800034c0     libForceEarlyReturnTest.obj
 0002:000004e0       ??_C@_0BJ@HPCAOILC@JVMTI_ERROR_INVALID_SLOT@ 00000001800034e0     libForceEarlyReturnTest.obj
 0002:00000500       ??_C@_0BG@CHILOPNI@JVMTI_ERROR_DUPLICATE@ 0000000180003500     libForceEarlyReturnTest.obj
 0002:00000518       ??_C@_0BG@DIEMLHKM@JVMTI_ERROR_NOT_FOUND@ 0000000180003518     libForceEarlyReturnTest.obj
 0002:00000530       ??_C@_0BM@NHMCKHOB@JVMTI_ERROR_INVALID_MONITOR@ 0000000180003530     libForceEarlyReturnTest.obj
 0002:00000550       ??_C@_0BO@PPEDAJGL@JVMTI_ERROR_NOT_MONITOR_OWNER@ 0000000180003550     libForceEarlyReturnTest.obj
 0002:00000570       ??_C@_0BG@FCAIPEID@JVMTI_ERROR_INTERRUPT@ 0000000180003570     libForceEarlyReturnTest.obj
 0002:00000588       ??_C@_0CB@EGDBNKOI@JVMTI_ERROR_INVALID_CLASS_FORMA@ 0000000180003588     libForceEarlyReturnTest.obj
 0002:000005b0       ??_C@_0CG@DGKOGIAL@JVMTI_ERROR_CIRCULAR_CLASS_DEFI@ 00000001800035b0     libForceEarlyReturnTest.obj
 0002:000005d8       ??_C@_0BP@ICEALPKC@JVMTI_ERROR_FAILS_VERIFICATION@ 00000001800035d8     libForceEarlyReturnTest.obj
 0002:000005f8       ??_C@_0DC@JDACLMIO@JVMTI_ERROR_UNSUPPORTED_REDEFIN@ 00000001800035f8     libForceEarlyReturnTest.obj
 0002:00000630       ??_C@_0DE@GKDKNOMJ@JVMTI_ERROR_UNSUPPORTED_REDEFIN@ 0000000180003630     libForceEarlyReturnTest.obj
 0002:00000668       ??_C@_0BO@LAFKIOG@JVMTI_ERROR_INVALID_TYPESTATE@ 0000000180003668     libForceEarlyReturnTest.obj
 0002:00000688       ??_C@_0DH@INDGCLLB@JVMTI_ERROR_UNSUPPORTED_REDEFIN@ 0000000180003688     libForceEarlyReturnTest.obj
 0002:000006c0       ??_C@_0DE@NHEOMMGI@JVMTI_ERROR_UNSUPPORTED_REDEFIN@ 00000001800036c0     libForceEarlyReturnTest.obj
 0002:000006f8       ??_C@_0CA@EKPNJOEP@JVMTI_ERROR_UNSUPPORTED_VERSION@ 00000001800036f8     libForceEarlyReturnTest.obj
 0002:00000718       ??_C@_0BN@OFFMAHHL@JVMTI_ERROR_NAMES_DONT_MATCH@ 0000000180003718     libForceEarlyReturnTest.obj
 0002:00000738       ??_C@_0DN@HHBBLAKE@JVMTI_ERROR_UNSUPPORTED_REDEFIN@ 0000000180003738     libForceEarlyReturnTest.obj
 0002:00000778       ??_C@_0DO@HMBGBGNA@JVMTI_ERROR_UNSUPPORTED_REDEFIN@ 0000000180003778     libForceEarlyReturnTest.obj
 0002:000007b8       ??_C@_0BP@PBECGKHJ@JVMTI_ERROR_UNMODIFIABLE_CLASS@ 00000001800037b8     libForceEarlyReturnTest.obj
 0002:000007d8       ??_C@_0BK@CANILEHF@JVMTI_ERROR_NOT_AVAILABLE@ 00000001800037d8     libForceEarlyReturnTest.obj
 0002:000007f8       ??_C@_0CE@INJKMEFK@JVMTI_ERROR_MUST_POSSESS_CAPABI@ 00000001800037f8     libForceEarlyReturnTest.obj
 0002:00000820       ??_C@_0BJ@LBFPFPDM@JVMTI_ERROR_NULL_POINTER@ 0000000180003820     libForceEarlyReturnTest.obj
 0002:00000840       ??_C@_0BP@CHJPNNEM@JVMTI_ERROR_ABSENT_INFORMATION@ 0000000180003840     libForceEarlyReturnTest.obj
 0002:00000860       ??_C@_0BP@OMFMNLC@JVMTI_ERROR_INVALID_EVENT_TYPE@ 0000000180003860     libForceEarlyReturnTest.obj
 0002:00000880       ??_C@_0BN@BIBNPHHO@JVMTI_ERROR_ILLEGAL_ARGUMENT@ 0000000180003880     libForceEarlyReturnTest.obj
 0002:000008a0       ??_C@_0BK@KKNDHDCE@JVMTI_ERROR_NATIVE_METHOD@ 00000001800038a0     libForceEarlyReturnTest.obj
 0002:000008c0       ??_C@_0BK@PMKCFHAE@JVMTI_ERROR_OUT_OF_MEMORY@ 00000001800038c0     libForceEarlyReturnTest.obj
 0002:000008e0       ??_C@_0BK@NNJBDMNB@JVMTI_ERROR_ACCESS_DENIED@ 00000001800038e0     libForceEarlyReturnTest.obj
 0002:00000900       ??_C@_0BI@GHECLMNC@JVMTI_ERROR_WRONG_PHASE@ 0000000180003900     libForceEarlyReturnTest.obj
 0002:00000918       ??_C@_0BF@OLIHJOII@JVMTI_ERROR_INTERNAL@ 0000000180003918     libForceEarlyReturnTest.obj
 0002:00000930       ??_C@_0BO@EOHGKJHI@JVMTI_ERROR_UNATTACHED_THREAD@ 0000000180003930     libForceEarlyReturnTest.obj
 0002:00000950       ??_C@_0CA@LKHFDACL@JVMTI_ERROR_INVALID_ENVIRONMENT@ 0000000180003950     libForceEarlyReturnTest.obj
 0002:00000970       ??_C@_0BA@MMFHLOKK@?$DMunknown?5error?$DO@ 0000000180003970     libForceEarlyReturnTest.obj
 0002:00000980       ??_C@_0EI@KKLANDNF@Breakpoint?3?5Failed?5with?5wrong?5l@ 0000000180003980     libForceEarlyReturnTest.obj
 0002:000009c8       ??_C@_0DI@CMPIBDC@Breakpoint?3?5In?5method?5TestTask?4@ 00000001800039c8     libForceEarlyReturnTest.obj
 0002:00000a00       ??_C@_0DH@DIPDMAEA@Breakpoint?3?5In?5method?5TestTask?4@ 0000000180003a00     libForceEarlyReturnTest.obj
 0002:00000a38       ??_C@_0CI@CABNHNCA@Breakpoint?3?5Failed?5in?5JVMTI?5Get@ 0000000180003a38     libForceEarlyReturnTest.obj
 0002:00000a60       ??_C@_0CM@JHEGJDLK@Breakpoint?3?5Failed?5in?5JVMTI?5Cle@ 0000000180003a60     libForceEarlyReturnTest.obj
 0002:00000a90       ??_C@_0CL@HCCDPLK@Breakpoint?3?5Failed?5in?5JVMTI?5Get@ 0000000180003a90     libForceEarlyReturnTest.obj
 0002:00000ac0       ??_C@_0DI@GAJJPHJI@Breakpoint?3?5Self?5early?5return?5f@ 0000000180003ac0     libForceEarlyReturnTest.obj
 0002:00000af8       ??_C@_0DL@NKKPDFLF@Breakpoint?3?5ForceEarlyReturnObj@ 0000000180003af8     libForceEarlyReturnTest.obj
 0002:00000b38       ??_C@_0CN@BIBCGBOC@Breakpoint?3?5Failed?5in?5ForceEarl@ 0000000180003b38     libForceEarlyReturnTest.obj
 0002:00000b68       ??_C@_0CN@HHMPLKB@Breakpoint?3?5In?5method?5TestTask?4@ 0000000180003b68     libForceEarlyReturnTest.obj
 0002:00000b98       ??_C@_0M@PEALHFHB@Agent?5init?6@ 0000000180003b98     libForceEarlyReturnTest.obj
 0002:00000ba8       ??_C@_0BP@JDPNKEIH@Agent?5init?3?5Failed?5in?5GetEnv?$CB?6@ 0000000180003ba8     libForceEarlyReturnTest.obj
 0002:00000bc8       ??_C@_0DJ@NBPJDIMI@Agent?5init?3?5Failed?5in?5GetPotent@ 0000000180003bc8     libForceEarlyReturnTest.obj
 0002:00000c08       ??_C@_0DA@JFMHIKLD@Agent?5init?3?5Failed?5in?5AddCapabi@ 0000000180003c08     libForceEarlyReturnTest.obj
 0002:00000c38       ??_C@_0DA@HAPJLIDB@Agent?5init?3?5Failed?5in?5GetCapabi@ 0000000180003c38     libForceEarlyReturnTest.obj
 0002:00000c68       ??_C@_0DJ@INFOBIKA@Agent?5init?3?5Failed?3?5Breakpoint?5@ 0000000180003c68     libForceEarlyReturnTest.obj
 0002:00000ca8       ??_C@_0DC@FCGCPGJF@Agent?5init?3?5Failed?5in?5SetEventC@ 0000000180003ca8     libForceEarlyReturnTest.obj
 0002:00000ce0       ??_C@_0BE@GGOHGOCG@Raw?5monitor?5to?5test@ 0000000180003ce0     libForceEarlyReturnTest.obj
 0002:00000cf8       ??_C@_0BM@IDJGICLI@Main?3?5prepareAgent?5started?6@ 0000000180003cf8     libForceEarlyReturnTest.obj
 0002:00000d18       ??_C@_0DP@KMAPEEIK@prepareAgent?3?5Failed?5as?5JVMTI?5c@ 0000000180003d18     libForceEarlyReturnTest.obj
 0002:00000d58       ??_C@_0CI@PEDDEGJK@?$CIZLjava?1lang?1String?$DL?$CJLjava?1lang@ 0000000180003d58     libForceEarlyReturnTest.obj
 0002:00000d80       ??_C@_01HMGJMAIH@B@        0000000180003d80     libForceEarlyReturnTest.obj
 0002:00000d90       ??_C@_0EB@DNGPDOEE@prepareAgent?3?5Failed?5to?5find?5Me@ 0000000180003d90     libForceEarlyReturnTest.obj
 0002:00000dd8       ??_C@_0CM@LKEDMPML@prepareAgent?3?5Failed?5in?5JVMTI?5S@ 0000000180003dd8     libForceEarlyReturnTest.obj
 0002:00000e08       ??_C@_0BN@EHAFOC@Main?3?5prepareAgent?5finished?6@ 0000000180003e08     libForceEarlyReturnTest.obj
 0002:00000e28       ??_C@_0BF@CHNHCBN@Main?3?5suspendThread?6@ 0000000180003e28     libForceEarlyReturnTest.obj
 0002:00000e40       ??_C@_0BE@NBLNCOLL@Main?3?5resumeThread?6@ 0000000180003e40     libForceEarlyReturnTest.obj
 0002:00000e60       ??_C@_0EF@FLJJHDFD@Main?3?5forceEarlyReturn?3?5ForceEa@ 0000000180003e60     libForceEarlyReturnTest.obj
 0002:00000eb0       ??_C@_0EE@IBBKIDKE@Main?3?5forceEarlyReturn?3?5ForceEa@ 0000000180003eb0     libForceEarlyReturnTest.obj
 0002:00000f00       ??_C@_0EH@OHACMCIE@Main?3?5forceEarlyReturn?3?5ForceEa@ 0000000180003f00     libForceEarlyReturnTest.obj
 0002:00000f48       ??_C@_0BK@FNGEELHP@Main?3?5ensureAtBreakpoint?6@ 0000000180003f48     libForceEarlyReturnTest.obj
 0002:00000f68       ??_C@_0BK@OIBCOPKF@Main?3?5notifyAtBreakpoint?6@ 0000000180003f68     libForceEarlyReturnTest.obj
 0002:00000f90       ??_C@_1EC@JIJBPKFM@?$AAa?$AAp?$AAi?$AA?9?$AAm?$AAs?$AA?9?$AAw?$AAi?$AAn?$AA?9?$AAc?$AAo?$AAr?$AAe@ 0000000180003f90     MSVCRT:thread_safe_statics.obj
 0002:00000fd8       ??_C@_1BK@MGMFAEKH@?$AAk?$AAe?$AAr?$AAn?$AAe?$AAl?$AA3?$AA2?$AA?4?$AAd?$AAl?$AAl@ 0000000180003fd8     MSVCRT:thread_safe_statics.obj
 0002:00000ff8       ??_C@_0BJ@JEBJOJFJ@SleepConditionVariableCS@ 0000000180003ff8     MSVCRT:thread_safe_statics.obj
 0002:00001018       ??_C@_0BJ@PGPPEPCC@WakeAllConditionVariable@ 0000000180004018     MSVCRT:thread_safe_statics.obj
 0002:00001038       _pDefaultRawDllMain        0000000180004038     MSVCRT:dll_dllmain.obj
 0002:00001038       _pRawDllMain               0000000180004038     MSVCRT:dll_dllmain.obj
 0002:00001040       __xmm@ffffffffffffffffffffffffffffffff 0000000180004040     MSVCRT:utility.obj
 0002:00001060       _load_config_used          0000000180004060     MSVCRT:loadcfg.obj
 0002:00001280       _tls_used                  0000000180004280     MSVCRT:tlssup.obj
 0002:000012a8       __volatile_metadata        00000001800042a8     <linker-defined>
 0002:00001640       __rtc_iaa                  0000000180004640     MSVCRT:initsect.obj
 0002:00001648       __rtc_izz                  0000000180004648     MSVCRT:initsect.obj
 0002:00001650       __rtc_taa                  0000000180004650     MSVCRT:initsect.obj
 0002:00001658       __rtc_tzz                  0000000180004658     MSVCRT:initsect.obj
 0002:00001660       _tls_start                 0000000180004660     MSVCRT:tlssup.obj
 0002:00001664       _Init_thread_epoch         0000000180004664     MSVCRT:thread_safe_statics.obj
 0002:00001668       _tls_end                   0000000180004668     MSVCRT:tlssup.obj
 0002:00001a2c       __IMPORT_DESCRIPTOR_KERNEL32 0000000180004a2c     kernel32:KERNEL32.dll
 0002:00001a40       __IMPORT_DESCRIPTOR_VCRUNTIME140 0000000180004a40     vcruntime:VCRUNTIME140.dll
 0002:00001a54       __IMPORT_DESCRIPTOR_api-ms-win-crt-stdio-l1-1-0 0000000180004a54     ucrt:api-ms-win-crt-stdio-l1-1-0.dll
 0002:00001a68       __IMPORT_DESCRIPTOR_api-ms-win-crt-runtime-l1-1-0 0000000180004a68     ucrt:api-ms-win-crt-runtime-l1-1-0.dll
 0002:00001a7c       __NULL_IMPORT_DESCRIPTOR   0000000180004a7c     kernel32:KERNEL32.dll
 0003:00000000       _Init_global_epoch         0000000180005000     MSVCRT:thread_safe_statics.obj
 0003:00000010       __security_cookie          0000000180005010     MSVCRT:gs_cookie.obj
 0003:00000018       __security_cookie_complement 0000000180005018     MSVCRT:gs_cookie.obj
 0003:00000020       __scrt_native_dllmain_reason 0000000180005020     MSVCRT:utility.obj
 0003:00000028       __isa_available            0000000180005028     MSVCRT:cpu_disp.obj
 0003:0000002c       __isa_enabled              000000018000502c     MSVCRT:cpu_disp.obj
 0003:00000030       __memset_fast_string_threshold 0000000180005030     MSVCRT:cpu_disp.obj
 0003:00000038       __memset_nt_threshold      0000000180005038     MSVCRT:cpu_disp.obj
 0003:00000040       __scrt_ucrt_dll_is_in_use  0000000180005040     MSVCRT:ucrt_stubs.obj
 0003:00000050       ?_OptionsStorage@?1??__local_stdio_printf_options@@9@4_KA 0000000180005050     libForceEarlyReturnTest.obj
 0003:00000210       _tls_index                 0000000180005210     MSVCRT:tlssup.obj
 0003:00000218       __scrt_current_native_startup_state 0000000180005218     MSVCRT:utility.obj
 0003:00000220       __scrt_native_startup_lock 0000000180005220     MSVCRT:utility.obj
 0003:00000260       __scrt_debugger_hook_flag  0000000180005260     MSVCRT:utility_desktop.obj
 0003:000007e0       ?__type_info_root_node@@3U__type_info_node@@A 00000001800057e0     MSVCRT:tncleanup.obj
 0003:000007f0       ?_OptionsStorage@?1??__local_stdio_scanf_options@@9@4_KA 00000001800057f0     MSVCRT:default_local_stdio_options.obj
 0003:000007f8       __favor                    00000001800057f8     MSVCRT:cpu_disp.obj
 0003:00000800       __dyn_tls_init_callback    0000000180005800     <common>

 entry point at        0001:00001030

 Static symbols

 0000:ffff8000       .debug$S                   0000000180000000     ForceEarlyReturnTest.exp
 0000:ffff8000       .debug$S                   0000000180000000     vcruntime:VCRUNTIME140.dll
 0000:ffff8000       .debug$S                   0000000180000000     vcruntime:VCRUNTIME140.dll
 0000:ffff8000       .debug$S                   0000000180000000     vcruntime:VCRUNTIME140.dll
 0000:ffff8000       .debug$S                   0000000180000000     vcruntime:VCRUNTIME140.dll
 0000:ffff8000       .debug$S                   0000000180000000     vcruntime:VCRUNTIME140.dll
 0000:ffff8000       .debug$S                   0000000180000000     vcruntime:VCRUNTIME140.dll
 0000:ffff8000       .debug$S                   0000000180000000     ucrt:api-ms-win-crt-runtime-l1-1-0.dll
 0000:ffff8000       .debug$S                   0000000180000000     ucrt:api-ms-win-crt-runtime-l1-1-0.dll
 0000:ffff8000       .debug$S                   0000000180000000     ucrt:api-ms-win-crt-runtime-l1-1-0.dll
 0000:ffff8000       .debug$S                   0000000180000000     ucrt:api-ms-win-crt-runtime-l1-1-0.dll
 0000:ffff8000       .debug$S                   0000000180000000     ucrt:api-ms-win-crt-runtime-l1-1-0.dll
 0000:ffff8000       .debug$S                   0000000180000000     ucrt:api-ms-win-crt-runtime-l1-1-0.dll
 0000:ffff8000       .debug$S                   0000000180000000     ucrt:api-ms-win-crt-runtime-l1-1-0.dll
 0000:ffff8000       .debug$S                   0000000180000000     ucrt:api-ms-win-crt-runtime-l1-1-0.dll
 0000:ffff8000       .debug$S                   0000000180000000     ucrt:api-ms-win-crt-runtime-l1-1-0.dll
 0000:ffff8000       .debug$S                   0000000180000000     ucrt:api-ms-win-crt-runtime-l1-1-0.dll
 0000:ffff8000       .debug$S                   0000000180000000     ucrt:api-ms-win-crt-runtime-l1-1-0.dll
 0000:ffff8000       .debug$S                   0000000180000000     ucrt:api-ms-win-crt-runtime-l1-1-0.dll
 0000:ffff8000       .debug$S                   0000000180000000     ucrt:api-ms-win-crt-stdio-l1-1-0.dll
 0000:ffff8000       .debug$S                   0000000180000000     ucrt:api-ms-win-crt-stdio-l1-1-0.dll
 0000:ffff8000       .debug$S                   0000000180000000     ucrt:api-ms-win-crt-stdio-l1-1-0.dll
 0000:ffff8000       .debug$S                   0000000180000000     ucrt:api-ms-win-crt-string-l1-1-0.dll
 0000:ffff8000       .debug$S                   0000000180000000     ucrt:api-ms-win-crt-string-l1-1-0.dll
 0000:ffff8000       .debug$S                   0000000180000000     ucrt:api-ms-win-crt-string-l1-1-0.dll
 0000:ffff8000       .debug$S                   0000000180000000     ucrt:api-ms-win-crt-string-l1-1-0.dll
 0002:ffffd000       .idata$6                   0000000180000000     ucrt:api-ms-win-crt-string-l1-1-0.dll
 0000:ffff8000       .debug$S                   0000000180000000     kernel32:KERNEL32.dll
 0000:ffff8000       .debug$S                   0000000180000000     kernel32:KERNEL32.dll
 0000:ffff8000       .debug$S                   0000000180000000     kernel32:KERNEL32.dll
 0000:ffff8000       .debug$S                   0000000180000000     kernel32:KERNEL32.dll
 0000:ffff8000       .debug$S                   0000000180000000     kernel32:KERNEL32.dll
 0000:ffff8000       .debug$S                   0000000180000000     kernel32:KERNEL32.dll
 0000:ffff8000       .debug$S                   0000000180000000     kernel32:KERNEL32.dll
 0000:ffff8000       .debug$S                   0000000180000000     kernel32:KERNEL32.dll
 0000:ffff8000       .debug$S                   0000000180000000     kernel32:KERNEL32.dll
 0000:ffff8000       .debug$S                   0000000180000000     kernel32:KERNEL32.dll
 0000:ffff8000       .debug$S                   0000000180000000     kernel32:KERNEL32.dll
 0000:ffff8000       .debug$S                   0000000180000000     kernel32:KERNEL32.dll
 0000:ffff8000       .debug$S                   0000000180000000     kernel32:KERNEL32.dll
 0000:ffff8000       .debug$S                   0000000180000000     kernel32:KERNEL32.dll
 0000:ffff8000       .debug$S                   0000000180000000     kernel32:KERNEL32.dll
 0000:ffff8000       .debug$S                   0000000180000000     kernel32:KERNEL32.dll
 0000:ffff8000       .debug$S                   0000000180000000     kernel32:KERNEL32.dll
 0000:ffff8000       .debug$S                   0000000180000000     kernel32:KERNEL32.dll
 0000:ffff8000       .debug$S                   0000000180000000     kernel32:KERNEL32.dll
 0000:ffff8000       .debug$S                   0000000180000000     kernel32:KERNEL32.dll
 0000:ffff8000       .debug$S                   0000000180000000     kernel32:KERNEL32.dll
 0000:ffff8000       .debug$S                   0000000180000000     kernel32:KERNEL32.dll
 0000:ffff8000       .debug$S                   0000000180000000     kernel32:KERNEL32.dll
 0000:ffff8000       .debug$S                   0000000180000000     kernel32:KERNEL32.dll
 0000:ffff8000       .debug$S                   0000000180000000     kernel32:KERNEL32.dll
 0000:ffff8000       .debug$S                   0000000180000000     kernel32:KERNEL32.dll
 0000:ffff8000       .debug$S                   0000000180000000     kernel32:KERNEL32.dll
 0000:ffff8000       .debug$S                   0000000180000000     kernel32:KERNEL32.dll
 0001:000002c4       ?check_jvmti_status@@YAXPEAUJNIEnv_@@W4jvmtiError@@PEBD@Z 00000001800012c4 f   libForceEarlyReturnTest.obj
 0001:00000504       Breakpoint                 0000000180001504 f   libForceEarlyReturnTest.obj
 0001:00000be4       ?__scrt_initialize_thread_safe_statics@@YAHXZ 0000000180001be4 f   MSVCRT:thread_safe_statics.obj
 0001:00000cb4       ?__scrt_uninitialize_thread_safe_statics@@YAXXZ 0000000180001cb4 f   MSVCRT:thread_safe_statics.obj
 0001:00000ce0       $$000000                   0000000180001ce0     MSVCRT:amdsecgs.obj
 0001:00000d10       ?dllmain_crt_dispatch@@YAHQEAUHINSTANCE__@@KQEAX@Z 0000000180001d10 f   MSVCRT:dll_dllmain.obj
 0001:00000d60       ?dllmain_crt_process_attach@@YAHQEAUHINSTANCE__@@QEAX@Z 0000000180001d60 f   MSVCRT:dll_dllmain.obj
 0001:00000e78       ?dllmain_crt_process_detach@@YAH_N@Z 0000000180001e78 f   MSVCRT:dll_dllmain.obj
 0001:00000efc       ?dllmain_dispatch@@YAHQEAUHINSTANCE__@@KQEAX@Z 0000000180001efc f   MSVCRT:dll_dllmain.obj
 0001:00001650       capture_previous_context   0000000180002650 f   MSVCRT:gs_report.obj
 0001:00001a80       $$000000                   0000000180002a80     MSVCRT:guard_dispatch.obj
 0001:00001aa0       $$000000                   0000000180002aa0     MSVCRT:guard_xfg_dispatch.obj
 0001:00001ab6       ?fin$0@?0??dllmain_crt_process_attach@@YAHQEAUHINSTANCE__@@QEAX@Z@4HA 0000000180002ab6 f   MSVCRT:dll_dllmain.obj
 0001:00001acd       ?fin$0@?0??dllmain_crt_process_detach@@YAH_N@Z@4HA 0000000180002acd f   MSVCRT:dll_dllmain.obj
 0001:00001ae6       ?fin$1@?0??dllmain_crt_process_detach@@YAH_N@Z@4HA 0000000180002ae6 f   MSVCRT:dll_dllmain.obj
 0001:00001afa       ?filt$0@?0??dllmain_dispatch@@YAHQEAUHINSTANCE__@@KQEAX@Z@4HA 0000000180002afa f   MSVCRT:dll_dllmain.obj
 0001:00001b30       __scrt_is_nonwritable_in_current_image$filt$0 0000000180002b30 f   MSVCRT:utility.obj
 0002:000001a8       ?__scrt_initialize_tss_var@@3P6AHXZEA 00000001800031a8     MSVCRT:thread_safe_statics.obj
 0002:00001050       GS_ExceptionPointers       0000000180004050     MSVCRT:gs_report.obj
 0002:00001670       $unwind$printf             0000000180004670     libForceEarlyReturnTest.obj
 0002:0000167c       $unwind$?check_jvmti_status@@YAXPEAUJNIEnv_@@W4jvmtiError@@PEBD@Z 000000018000467c     libForceEarlyReturnTest.obj
 0002:0000168c       $unwind$?create_raw_monitor@@YAPEAU_jrawMonitorID@@PEAU_jvmtiEnv@@PEBD@Z 000000018000468c     libForceEarlyReturnTest.obj
 0002:0000168c       $unwind$__scrt_initialize_default_local_stdio_options 000000018000468c     MSVCRT:default_local_stdio_options.obj
 0002:0000168c       $unwind$?dllmain_crt_dispatch@@YAHQEAUHINSTANCE__@@KQEAX@Z 000000018000468c     MSVCRT:dll_dllmain.obj
 0002:0000168c       $unwind$DllMain            000000018000468c     MSVCRT:dll_dllmain_stub.obj
 0002:0000168c       $unwind$?__scrt_uninitialize_thread_safe_statics@@YAXXZ 000000018000468c     MSVCRT:thread_safe_statics.obj
 0002:0000168c       $unwind$__scrt_acquire_startup_lock 000000018000468c     MSVCRT:utility.obj
 0002:0000168c       $unwind$__scrt_dllmain_after_initialize_c 000000018000468c     MSVCRT:utility.obj
 0002:0000168c       $unwind$__scrt_dllmain_before_initialize_c 000000018000468c     MSVCRT:utility.obj
 0002:0000168c       $unwind$__scrt_dllmain_crt_thread_attach 000000018000468c     MSVCRT:utility.obj
 0002:0000168c       $unwind$__scrt_dllmain_crt_thread_detach 000000018000468c     MSVCRT:utility.obj
 0002:0000168c       $unwind$__scrt_dllmain_uninitialize_c 000000018000468c     MSVCRT:utility.obj
 0002:0000168c       $unwind$__scrt_dllmain_uninitialize_critical 000000018000468c     MSVCRT:utility.obj
 0002:0000168c       $unwind$atexit             000000018000468c     MSVCRT:utility.obj
 0002:00001694       $unwind$Breakpoint         0000000180004694     libForceEarlyReturnTest.obj
 0002:000016a8       $unwind$Agent_Initialize   00000001800046a8     libForceEarlyReturnTest.obj
 0002:000016a8       $unwind$Java_ForceEarlyReturnTest_prepareAgent 00000001800046a8     libForceEarlyReturnTest.obj
 0002:000016a8       $unwind$Java_ForceEarlyReturnTest_resumeThread 00000001800046a8     libForceEarlyReturnTest.obj
 0002:000016a8       $unwind$Java_ForceEarlyReturnTest_suspendThread 00000001800046a8     libForceEarlyReturnTest.obj
 0002:000016a8       $unwind$_RTC_Initialize    00000001800046a8     MSVCRT:initsect.obj
 0002:000016a8       $unwind$_RTC_Terminate     00000001800046a8     MSVCRT:initsect.obj
 0002:000016a8       $unwind$?__scrt_initialize_thread_safe_statics@@YAHXZ 00000001800046a8     MSVCRT:thread_safe_statics.obj
 0002:000016b4       $unwind$Java_ForceEarlyReturnTest_forceEarlyReturnI 00000001800046b4     libForceEarlyReturnTest.obj
 0002:000016b4       $unwind$Java_ForceEarlyReturnTest_forceEarlyReturnO 00000001800046b4     libForceEarlyReturnTest.obj
 0002:000016b4       $unwind$Java_ForceEarlyReturnTest_forceEarlyReturnV 00000001800046b4     libForceEarlyReturnTest.obj
 0002:000016b4       $unwind$__raise_securityfailure 00000001800046b4     MSVCRT:gs_report.obj
 0002:000016b4       $unwind$__scrt_initialize_crt 00000001800046b4     MSVCRT:utility.obj
 0002:000016b4       $unwind$__scrt_initialize_onexit_tables 00000001800046b4     MSVCRT:utility.obj
 0002:000016b4       $unwind$__scrt_release_startup_lock 00000001800046b4     MSVCRT:utility.obj
 0002:000016b4       $unwind$__scrt_uninitialize_crt 00000001800046b4     MSVCRT:utility.obj
 0002:000016b4       $unwind$_onexit            00000001800046b4     MSVCRT:utility.obj
 0002:000016bc       $unwind$Java_ForceEarlyReturnTest_ensureAtBreakpoint 00000001800046bc     libForceEarlyReturnTest.obj
 0002:000016bc       $unwind$__scrt_dllmain_exception_filter 00000001800046bc     MSVCRT:utility.obj
 0002:000016d0       $unwind$Java_ForceEarlyReturnTest_notifyAtBreakpoint 00000001800046d0     libForceEarlyReturnTest.obj
 0002:000016d0       $unwind$_DllMainCRTStartup 00000001800046d0     MSVCRT:dll_dllmain.obj
 0002:000016e0       $xdatasym                  00000001800046e0     MSVCRT:amdsecgs.obj
 0002:000016e4       $unwind$?dllmain_crt_process_attach@@YAHQEAUHINSTANCE__@@QEAX@Z 00000001800046e4     MSVCRT:dll_dllmain.obj
 0002:00001720       $unwind$?fin$0@?0??dllmain_crt_process_attach@@YAHQEAUHINSTANCE__@@QEAX@Z@4HA 0000000180004720     MSVCRT:dll_dllmain.obj
 0002:00001720       $unwind$?fin$0@?0??dllmain_crt_process_detach@@YAH_N@Z@4HA 0000000180004720     MSVCRT:dll_dllmain.obj
 0002:00001720       $unwind$?fin$1@?0??dllmain_crt_process_detach@@YAH_N@Z@4HA 0000000180004720     MSVCRT:dll_dllmain.obj
 0002:00001728       $unwind$?dllmain_crt_process_detach@@YAH_N@Z 0000000180004728     MSVCRT:dll_dllmain.obj
 0002:0000177c       $unwind$?dllmain_dispatch@@YAHQEAUHINSTANCE__@@KQEAX@Z 000000018000477c     MSVCRT:dll_dllmain.obj
 0002:000017a4       $unwind$?filt$0@?0??dllmain_dispatch@@YAHQEAUHINSTANCE__@@KQEAX@Z@4HA 00000001800047a4     MSVCRT:dll_dllmain.obj
 0002:000017ac       $unwind$__scrt_is_nonwritable_in_current_image 00000001800047ac     MSVCRT:utility.obj
 0002:000017cc       $unwind$__scrt_is_nonwritable_in_current_image$filt$0 00000001800047cc     MSVCRT:utility.obj
 0002:000017d4       $unwind$__scrt_fastfail    00000001800047d4     MSVCRT:utility_desktop.obj
 0002:000017e4       $unwind$__report_gsfailure 00000001800047e4     MSVCRT:gs_report.obj
 0002:000017ec       $unwind$capture_previous_context 00000001800047ec     MSVCRT:gs_report.obj
 0002:000017f8       $unwind$__security_init_cookie 00000001800047f8     MSVCRT:gs_support.obj
 0002:00001804       $unwind$__isa_available_init 0000000180004804     MSVCRT:cpu_disp.obj
 0002:00001818       $xdatasym                  0000000180004818     MSVCRT:guard_dispatch.obj
 0002:00001820       $xdatasym                  0000000180004820     MSVCRT:guard_xfg_dispatch.obj
 0002:00001830       .edata                     0000000180004830     ForceEarlyReturnTest.exp
 0002:00001858       rgpv                       0000000180004858     ForceEarlyReturnTest.exp
 0002:0000187c       rgszName                   000000018000487c     ForceEarlyReturnTest.exp
 0002:000018a0       rgwOrd                     00000001800048a0     ForceEarlyReturnTest.exp
 0002:000018b2       szName                     00000001800048b2     ForceEarlyReturnTest.exp
 0002:000018cb       $N00001                    00000001800048cb     ForceEarlyReturnTest.exp
 0002:000018d8       $N00002                    00000001800048d8     ForceEarlyReturnTest.exp
 0002:00001905       $N00003                    0000000180004905     ForceEarlyReturnTest.exp
 0002:00001931       $N00004                    0000000180004931     ForceEarlyReturnTest.exp
 0002:0000195d       $N00005                    000000018000495d     ForceEarlyReturnTest.exp
 0002:00001989       $N00006                    0000000180004989     ForceEarlyReturnTest.exp
 0002:000019b6       $N00007                    00000001800049b6     ForceEarlyReturnTest.exp
 0002:000019dd       $N00008                    00000001800049dd     ForceEarlyReturnTest.exp
 0002:00001a04       $N00009                    0000000180004a04     ForceEarlyReturnTest.exp
 0002:00001dda       .idata$6                   0000000180004dda     kernel32:KERNEL32.dll
 0002:00001e2a       .idata$6                   0000000180004e2a     vcruntime:VCRUNTIME140.dll
 0002:00001f42       .idata$6                   0000000180004f42     ucrt:api-ms-win-crt-stdio-l1-1-0.dll
 0002:00001f62       .idata$6                   0000000180004f62     ucrt:api-ms-win-crt-runtime-l1-1-0.dll
 0003:00000058       jvmti                      0000000180005058     libForceEarlyReturnTest.obj
 0003:00000060       mid_B                      0000000180005060     libForceEarlyReturnTest.obj
 0003:00000068       monitor                    0000000180005068     libForceEarlyReturnTest.obj
 0003:00000070       bp_sync_reached            0000000180005070     libForceEarlyReturnTest.obj
 0003:00000078       ?caps@?1??Agent_Initialize@@9@4UjvmtiCapabilities@@A 0000000180005078     libForceEarlyReturnTest.obj
 0003:00000090       ?callbacks@?1??Agent_Initialize@@9@4UjvmtiEventCallbacks@@A 0000000180005090     libForceEarlyReturnTest.obj
 0003:000001c8       ?g_tss_cv@@3U_RTL_CONDITION_VARIABLE@@A 00000001800051c8     MSVCRT:thread_safe_statics.obj
 0003:000001d0       ?g_tss_event@@3PEAXEA      00000001800051d0     MSVCRT:thread_safe_statics.obj
 0003:000001d8       ?g_tss_mutex@@3U_RTL_CRITICAL_SECTION@@A 00000001800051d8     MSVCRT:thread_safe_statics.obj
 0003:00000200       ?g_sleep_condition_variable_cs@@3P6AHPEAU_RTL_CONDITION_VARIABLE@@PEAU_RTL_CRITICAL_SECTION@@K@ZEA 0000000180005200     MSVCRT:thread_safe_statics.obj
 0003:00000208       ?g_wake_all_condition_variable@@3P6AXPEAU_RTL_CONDITION_VARIABLE@@@ZEA 0000000180005208     MSVCRT:thread_safe_statics.obj
 0003:00000214       ?__proc_attached@@3HA      0000000180005214     MSVCRT:dll_dllmain.obj
 0003:00000228       ?is_initialized_as_dll@@3_NA 0000000180005228     MSVCRT:utility.obj
 0003:00000229       ?module_local_atexit_table_initialized@@3_NA 0000000180005229     MSVCRT:utility.obj
 0003:00000230       ?module_local_atexit_table@@3U_onexit_table_t@@A 0000000180005230     MSVCRT:utility.obj
 0003:00000248       ?module_local_at_quick_exit_table@@3U_onexit_table_t@@A 0000000180005248     MSVCRT:utility.obj
 0003:00000270       GS_ExceptionRecord         0000000180005270     MSVCRT:gs_report.obj
 0003:00000310       GS_ContextRecord           0000000180005310     MSVCRT:gs_report.obj
